:1000000012C02BC02AC029C028C027C026C025C0C6
:1000100024C0DDC022C021C020C01FC01EC01DC022
:100020001CC01BC01AC011241FBECFE5D4E0DEBF28
:10003000CDBF10E0A0E6B0E0ECEEF2E002C005902B
:100040000D92A036B107D9F710E0A0E6B0E001C0EC
:100050001D92A536B107E1F75FC0D2CFCF93DF93F2
:10006000CDB7DEB721970FB6F894DEBF0FBECDBF78
:100070001982949A959A969A979AC09A8C988D9884
:100080008E988F98B898B998C198BA9AC29884E611
:100090008A95F1F7849903C0898181608983859964
:1000A00003C0898184608983869903C089818061C6
:1000B0008983879903C0898180648983B99AC198AB
:1000C000BA98C29884E68A95F1F7849903C0898129
:1000D00082608983859903C0898188608983869934
:1000E00003C0898180628983879903C08981806880
:1000F00089838981992721960FB6F894DEBF0FBEB8
:10010000CDBFDF91CF91089510BC89B908955F9B51
:10011000FECF8CB199270895CFE5D4E0DEBFCDBFE7
:100120009DDF182F8FEF84BB8AE081BB12BA80E07D
:1001300091E0909363008093620080E280930101DC
:1001400080E38093020180E18093030188E1809342
:10015000040188E0809305018CE08093060184E02F
:100160008093070184E2809308018BE48093600010
:1001700081E090E0C9DF91E09093610085E083BF6A
:1001800099BF7894103809F4FFCFC0E08099C0E09F
:10019000CF5FC236D8F3C0E0809BC0E0CF5FCC30E9
:1001A000D8F35F9B03C0CCB15F99FDCF80E18AB9E2
:1001B000C0E0ADDFCF5F1C17E0F7C0E0A8DF8093A1
:1001C0006000CAB9E2CF5D9BFECF8CB908957894E8
:1001D0001F920F920FB60F9211242F933F938F937C
:1001E0009F93EF93FF933FB7F89412BE2091600066
:1001F0002A3050F480916100E0916200F091630038
:10020000E80FF11D808185BB822F8A50853770F5FC
:10021000273428F0809164008A5F809364002F3136
:1002200028F0809164008E5F80936400822F880F95
:10023000835182BF809164008F5F809364008A3114
:10024000A8F01092640090916100E0916200F0913A
:100250006300E90FF11D808185BB892F8F5F80933B
:100260006100893018F081E080936100822F8F5700
:100270008C3008F415BA2B3868F1283C28F08091AE
:1002800064008A5F80936400263928F080916400BE
:100290008E5F80936400220F255122BF80916400FD
:1002A0008F5F809364008A31A8F01092640090916F
:1002B0006100E0916200F0916300E90FF11D80811F
:1002C00085BB892F815080936100882319F488E0D1
:1002D000809361003FBFFF91EF919F918F913F917C
:0C02E0002F910F900FBE0F901F901895EB
:00000001FF
